:020000040000FA
:10000000012807309F00831605118117FF308600F5
:1000100083128B138B150608A300A3092312A312C6
:100020002313A3132308A307A30723084720A4002F
:10003000800603194228A30A23084720A500A30A23
:1000400023084720A6002408A0002508A2002608AF
:10005000861B4228061F2F28861E2F28422838205C
:10006000051D3328362800000515232805112328EF
:10007000A00B3B283F28A100A10B3C283828A20B4D
:100080003F2808000B10630000008B130B28820729
:10009000863482341034843480340F347B347C349E
:1000A0000F34723482340F346334913410345B343F
:1000B0004734113409346E34B9340A347134983405
:1000C0000A34CA3483345634493411340034003489
:1000D0000034003400340034003400340034003480
:1000E0000034003400340034003400340034003470
:02400E00013F70
:00000001FF
